:10000000B5C0000036C20000CFC00000CDC0000067
:10001000CBC00000C9C00000C7C00000C5C00000C0
:10002000C3C00000C1C000000C94EE0EBDC00000B3
:10003000BBC00000B9C00000B7C00000B5C00000E0
:10004000B3C000003AC20000AFC00000ADC0000065
:10005000ABC0000079C30000A7C00000A5C000002D
:10006000A3C00000A1C000009FC000009DC0000010
:100070009BC0000099C0000097C0000095C0000020
:1000800072C2000091C000008FC000008DC000004F
:100090008BC0000089C0000026034C0055004600BC
:1000A00041002000580050004C00410049004E0023
:1000B00020004200720069006400670065000000D3
:1000C00018034400650061006E00200043006100D9
:1000D0006D0065007200610000000403090409025C
:1000E0003E0002010080320904000001020201000A
:1000F000052400100104240206052406000107055A
:1001000082030800FF09040100020A00000007053D
:1001100004021000050705830210000512011001FA
:1001200002000010EB034B2001000102DC01180368
:1001300041005600520049005300500020006D005D
:100140006B004900490000000C03410054004D00C1
:1001500045004C0000000403090412011001FF00D7
:100160000010EB03042100020102030111241FBE51
:10017000CFEFD0E2DEBFCDBF11E0A0E0B1E0E2E919
:10018000F5E200E00BBF02C007900D92AC3BB10757
:10019000D9F722E0ACEBB1E001C01D92AA3EB20754
:1001A000E1F7C7D00C94C7122BCF95B1809590641E
:1001B000892385B908958EB3843069F4F6D382E03B
:1001C0008093E9008091E80082FF05C080E4EDDFC4
:1001D000E7D280E0EACF08950F931F93CF93DF9388
:1001E0008EB3843009F06DC08FB7F8942091CC02A3
:1001F0003091CD028FBF8091CA029091CB02281717
:10020000390709F180E091E00E94A91197FD1BC018
:10021000E2ECF2E0A081B1818C9380819181019622
:1002200091838083268137818217930721F484810B
:100230009581918380832FB7F89482859385019669
:10024000938782872FBF8FB7F894C091D802D0913F
:10025000D9028FBFA8990BC0C93CD10540F480E0FA
:1002600091E0DF91CF911F910F910C949411A89A76
:100270000EEC12E023C0E091D002F091D102608137
:1002800080E091E00E9442118111E9CFF801828162
:100290009381019693838283268137818217930706
:1002A00021F484819581938382832FB7F89482858A
:1002B00093850197938782872FBF21972097D9F63F
:1002C000CECFDF91CF911F910F91089584B7877F93
:1002D00084BF88E10FB6F8948093600010926000AC
:1002E0000FBE90E080E80FB6F89480936100909381
:1002F00061000FBE85B7806885BF85B7806885BF00
:100300008F9A8FE19EE40197F1F700C000008FB152
:100310008095881F8827881F8093BC0185B78F77B9
:1003200085BF85B78F7785BF8AD0269A2E9A0C9481
:10033000D30ECCDF80E439DF78948091BC01811149
:1003400002C04ADF01C037DF0E940211F6CFCF930F
:10035000DF931F92CDB7DEB78091BC01811135C00C
:1003600080E091E00E941D1195E095BDE2ECF2E085
:100370009FB7F8942DEB31E03183208333832283C0
:10038000358324832DE332E03783268340E850E031
:1003900051874087138612869FBFEEECF2E09FB72D
:1003A000F8942DE332E03183208333832283358335
:1003B00024832DEB32E037832683518740871386D1
:1003C00012869FBF89833BD007C042E360E882E08A
:1003D0000E94F00D8983CDD18981882311F080E0BE
:1003E00001C080E40F90DF91CF91DFCE8091BC01FE
:1003F000811104C080E091E00C94DA11089580E44A
:10040000D4CE80E4D2CEFC0124893589468957892F
:1004100060E072E18AE790E00E948B12215031097E
:10042000309389002093880030939900209398009E
:1004300008957091BC01711101C0F2C030C1599A88
:10044000519A589A22E02093690081E08DBB80E4A4
:1004500093E0909389008093880090939900809313
:10046000980020936F002093710089E080939100A1
:1004700008951F920F920FB60F9211248F939F939E
:1004800088E08093BD0280918800909189009695C4
:10049000879591958195910990938500809384002B
:1004A000489904C01DBA89E0809381009F918F9183
:1004B0000F900FBE0F901F9018951F920F920FB6BE
:1004C0000F9211240BB60F922F933F938F939F930C
:1004D000AF93BF93EF93FF9389B181702091BD02D9
:1004E000222371F09091BE0296959093BE02215006
:1004F0002093BD02882341F190689093BE0224C0EE
:100500001092810091E09CBB9DBB8823E9F0EEEC4A
:10051000F2E0A081B1818091BE028C9380819181B3
:10052000019691838083268137818217930721F476
:1005300084819581918380832FB7F89482859385F8
:100540000196938782872FBFFF91EF91BF91AF9163
:100550009F918F913F912F910F900BBE0F900FBEE7
:100560000F901F9018951F920F920FB60F921124A3
:100570000BB60F922F933F938F939F93AF93BF939D
:10058000EF93FF938091BF02882371F08091C002A6
:1005900080FF02C0599801C0599A86958093C00285
:1005A0008091BF0281502BC08091BD02811129C072
:1005B0002FB7F8948091CC029091CD022FBF892B58
:1005C00001F15998E2ECF2E0A281B3812D91B3835D
:1005D000A28386819781A817B90721F48481958128
:1005E000938382833FB7F89482859385019793879D
:1005F00082873FBF822F80958093C00289E08093DD
:10060000BF02FF91EF91BF91AF919F918F913F9169
:100610002F910F900BBE0F900FBE0F901F9018954B
:10062000D9011C92292F33272230310539F023308C
:10063000310549F02130310521F128C0EEE3F0E029
:100640008EED90E027C099278130910561F08230CE
:10065000910581F0892BD1F4EAEDF0E0E491F0E02E
:100660008AED90E017C0E0ECF0E0E491F0E080EC7F
:1006700090E010C0E8E9F0E0E491F0E088E990E073
:1006800009C0E2E1F0E08CE191E004C0E0E0F0E0DC
:1006900080E090E0DA018D939C93CF010895D90119
:1006A0001C92292F33272230310541F023303105A8
:1006B00061F02130310509F439C03DC082E08C93EE
:1006C000E0E2F0E089E391E03AC0992781309105BA
:1006D00089F01CF4892B39F02EC08230910589F005
:1006E000039749F515C0E6E5F1E0E491F0E086E511
:1006F00091E025C0E8E4F1E0E491F0E088E491E0E5
:100700001EC0EEE2F1E0E491F0E08EE291E017C06D
:10071000E0911B01F0E082E390E090932A01809346
:10072000290182E08C938BE191E009C0E2E1F0E0E5
:100730008AE591E004C0E0E0F0E080E090E0DA01DA
:100740008D939C93CF01089578941F920F920FB6CA
:100750000F9211248F938AB5882321F08AB5815096
:100760008ABD01C015BC8F910F900FBE0F901F90D6
:100770001895EAE7F0E087EA80838298AEE7B0E078
:100780008C9184608C9382E480937C00808180646F
:1007900080838DE487BD82E084BD80936E00EAC0D3
:1007A0000F931F93CF93DF931F92CDB7DEB71091B6
:1007B000F10084E68ABD85E085BD163009F45AC093
:1007C00040F4113081F008F498C0143008F095C05E
:1007D00026C0103509F488C0113509F483C01A30D9
:1007E00009F08BC06DC08091E8008B778093E800A2
:1007F00082E08093E9008091EC0081608093EC00BE
:100800001093F1001092F1008AE08093F10040E033
:1008100050E06AE070E081EB91E0D4D787C00091AE
:10082000F100123011F46091F1008091E8008B77B3
:100830008093E80082E08093E9008091EC00816081
:100840008093EC001093F100802F6983C5D06981FB
:10085000123039F481FF0CC01092F100802FCCD0FF
:1008600065C080FF05C01092F100802FBDD05CC034
:1008700080EC5AC040E050E064E070E08BED92E024
:100880000E947E0C8091E8008B778093E80082E0E4
:100890008093E9008091EC0081608093EC0080916E
:1008A000DB029091DC02A091DD02B091DE02B7FF85
:1008B00003C081E08093DA0286E08093F1000FC0EC
:1008C0008091E8008B778093E80082E08093E900D4
:1008D0008091EC0081608093EC001093F100109205
:1008E000F10024C0EAD127C018D225C08091E800C9
:1008F0008B778093E8000E94620E8091F2009091C5
:10090000F3008034910591F38091E8008B77809318
:10091000E80082E08093E9008091EC0081608093A0
:10092000EC001093F10089EC8093F1008091E800D5
:100930008E778093E80015BC0E94620E82E080935F
:10094000E9008091EC008E7F8093EC000F90DF91A6
:10095000CF911F910F910895E9E5F1E090818917FA
:1009600039F0339691E0E737F907C1F7E0E0F0E0BE
:10097000CF010895CF93DF9380E090E00E94AD1205
:10098000D82F81E090E00E94AD12C82FDF3F21F008
:100990008EE9E2DFFC01D283CF3F21F088E9DCDF82
:1009A000FC01C283DF91CF91089584E9D5DFEAE7A6
:1009B000F0E02081206120834091780050917900FF
:1009C00062E3649F9001659F300D1124232F2695CB
:1009D0002695FC0122830895BFDF009719F0FC01E2
:1009E0008181089580E00895B7DF009719F0FC0138
:1009F0008281089580E008951F93CF93DF931F9223
:100A0000CDB7DEB7182F6983A7DF6981009789F01A
:100A1000FC0162831E3919F480E090E004C01839AB
:100A200041F481E090E00F90DF91CF911F910C9401
:100A3000B5120F90DF91CF911F9108959B01692FFF
:100A4000782F832F922F0895CF93DF93CDB7DEB702
:100A5000C750D1400FB6F894DEBF0FBECDBF40E007
:100A600050E067E070E0CE018F5F9E4FF9D6CE5F19
:100A7000DE4F688179818A819B81C250D140DEDF5F
:100A8000CE5FDE4F688379838A839B83C250D140D7
:100A9000CA5FDE4F8881C650D140C95FDE4F988162
:100AA000C750D140CA5FDE4F9883C650D140C95F5E
:100AB000DE4F8883C750D1408091E8008B778093C8
:100AC000E80082E08093E9008091EC0081608093EF
:100AD000EC008091C102CA5FDE4F28813981C65087
:100AE000D140811112C0CE5FDE4F688179818A8149
:100AF0009B81C250D140AE014F5F5F4FE8D3882346
:100B000011F080E00EC083E00CC0A901BE016F5F50
:100B10007F4FCE5FDE4F88819981C250D140D1D5C1
:100B2000EECF90E59093F10095E09093F1008093E3
:100B3000F10081110BC0CA5FDE4F68817981C65018
:100B4000D14040E050E0CE0101963CD68091E800D3
:100B50008E778093E800C95FDE4F0FB6F894DEBF52
:100B60000FBECDBFDF91CF910895AF92BF92CF92CC
:100B7000DF92EF92FF920F931F93CF93DF93CDB746
:100B8000DEB7C850D1400FB6F894DEBF0FBECDBF60
:100B900040E050E068E070E0CE01019661D66B81E4
:100BA0007C818D819E814ADF6B837C838D839E83D4
:100BB0007F8168856F83788740E050E0CE01099699
:100BC0004FD68F81988509968F739927892B39F491
:100BD0008091E8008B778093E8000E94620E8091FC
:100BE000E8008B778093E80082E08093E9008091B1
:100BF000EC0081608093EC008091C10281112EC0D5
:100C000029812150EB80FC800D811E812630A0F4CB
:100C100030E0F901E957FE4F8081F901E357FE4FBB
:100C20009081F901ED56FE4F6081F901E756FE4FC4
:100C30002081222359F103C066E293E28EE2AF8065
:100C4000B88429E0C22ED12CCC0EDD1E2A81482F7B
:100C5000892FB0D381110BC083E00AC04F81588522
:100C6000BE01675F7F4F8B819C8157D5F3CF80E0BA
:100C700090E59093F10094E09093F1008093F1005F
:100C80008091E8008E778093E80005C02985B8013F
:100C9000A70162D3DFCFC85FDE4F0FB6F894DEBF87
:100CA0000FBECDBFDF91CF911F910F91FF90EF90BD
:100CB000DF90CF90BF90AF900895CF93DF931F92B6
:100CC000CDB7DEB740E050E061E070E0CE010196C4
:100CD000C7D58091E8008B778093E80082E080930D
:100CE000E9008091EC0081608093EC008981809321
:100CF000C10281E58093F1008981813011F080E0AB
:100D000001C080EC8093F1008091E8008E778093A1
:100D1000E8000F90DF91CF910895CF93DF93CDB787
:100D2000DEB729970FB6F894DEBF0FBECDBF809116
:100D3000F100843009F492C040F4823079F108F077
:100D400049C0813009F02BC109C0863009F48AC03E
:100D500008F486C0873009F022C1CDC08091E80038
:100D60008B778093E80082E08093E9008091EC002B
:100D700081608093EC008091C102811102C01DD27C
:100D800005C0823011F44FD401C080E090E590930B
:100D9000F10091E09093F1008927FAC09091E8006A
:100DA0009B779093E8008093E9008091EC0081604C
:100DB0008093EC008091C102811102C045D201C034
:100DC00075D480E58093F10082E08093F100109269
:100DD000F100E0C040E050E065E070E0CE01019637
:100DE0003FD56A817B818C819D8128DE6A837B83EC
:100DF0008C839D838091E8008B778093E80082E06C
:100E00008093E9008091EC0081608093EC008091F8
:100E1000C102E981811114C0E150E83028F4F0E00A
:100E2000E158FE4F808101C080E04A815B816C8186
:100E30007D8135D3882311F080E00BC083E009C0A9
:100E4000E13011F480E101C084E16A817B819DD4AD
:100E5000F1CF90E59093F10093E098C086DE9FC0BB
:100E6000F3DD9DC040E050E061E070E0CE0101960E
:100E7000F7D48091E8008B778093E80082E080933C
:100E8000E9008091EC0081608093EC008091C102C8
:100E9000811112C0E981E150E23028F4F0E0E1561E
:100EA000FE4F808101C088E7BE016A5F7F4FD7D1C6
:100EB000882321F080E003C081E001C083E090E559
:100EC0009093F10096E09093F1008093F1008111EE
:100ED00061C08E819F81A885B985CD01AA27BB27D6
:100EE0008093F1008E819F81A885B9858093F10060
:100EF000892F99274DC08091F100833029F128F482
:100F0000813041F0823081F516C0843011F1853096
:100F100059F524C08091F1009091F1002091F100E9
:100F20003091F10030937B0120937C0190937D01FF
:100F300080937E0117C08091F1009091F100909311
:100F4000790180937A010EC08091F100809378013D
:100F500009C08091F1008093770104C08091F10075
:100F60008091F10080E001C081E09091E8009B77E2
:100F70009093E80092E09093E9009091EC009160EA
:100F80009093EC0090E59093F10097E09093F1003E
:100F90008093F1008091E8008E778093E800299695
:100FA0000FB6F894DEBF0FBECDBFDF91CF9108958D
:100FB0004D99FECF4D9BFECF4D99FECF5B9A539A34
:100FC0008091C9008F7E8093C9008091C90088609C
:100FD0008093C90081E08093DF0208958091C8006A
:100FE00086FFFCCF8091C80080648093C800809108
:100FF000C900877F8093C9008091C9008061809378
:10100000C90053985B981092DF0208958091DF0227
:101010008111E4DF80EC8093C8001092C900109227
:10102000CA008AB1877D8AB98BB1837D8BB9089557
:101030008091DF028111D2DF8091C800806C8093A3
:10104000C8001092C9001092CA008AB1877D8AB97F
:101050008BB1837D8BB924982C980895CF93DF931F
:101060001F92CDB7DEB79091DF02911103C0898343
:101070009FDF89819091C80095FFFCCF9091C800B7
:1010800090649093C8008093CE000F90DF91CF9131
:1010900008958091DF028111A1DF8091C80087FD52
:1010A00003C08AB58111F9CF8091CE000895809157
:1010B000DF02811101C07CDF8CE04D99FECF4D9B9A
:1010C000FECF4D99FECF8150C1F708951092DF02F7
:1010D000249A2C9887EC90E00197F1F700C000006B
:1010E0008AB188628AB9529881E090E09093CD00ED
:1010F0008093CC0088E08093C9008FE68093CA007B
:10110000D6DFD5CF1092DF028AB188628AB95298B1
:101110005B9A87EC90E00197F1F700C0000081E056
:1011200090E09093CD008093CC0088E08093C9003C
:101130008FE68093CA00BBDFBACF1F93CF93DF93B4
:1011400000D0CDB7DEB7182F862F79839A8386DF3C
:101150007981872F83DF812F81DF9A81892F0F90FB
:101160000F90DF91CF911F9179CF40917B015091EA
:101170007C0160917D0170917E01482BCB01BA0109
:10118000DCCF80E86BDF85DF9AB5992321F081FF02
:10119000F8CF81E0089580E008958BE65FDF8FE06F
:1011A000E4DF80E25BDF75DF9AB5992321F087FDEC
:1011B000F8CF81E0089580E00895BF92CF92DF924A
:1011C000EF92FF920F931F93CF93DF93CDB7DEB7CC
:1011D00028970FB6F894DEBF0FBECDBF93DF81EC2A
:1011E0003DDF89E53BDF82EC39DF82E037DF80EEEF
:1011F00035DF7E0189E0E80EF11C8E010F5F1F4F85
:1012000088E0D82EB02EC12EE1EAF1E0AB2DBC2D46
:101210008D2D01900D928A95E1F7F70182917F0162
:101220001DDFE016F10681F728960FB6F894DEBFB1
:101230000FBECDBFDF91CF911F910F91FF90EF9027
:10124000DF90CF90BF909DCF9CDF81EC07DF80E0E7
:1012500005DF81E803DF1DDF8111F7CFD7CE1F93B4
:10126000CF93DF93182FEB01188219821A821B8209
:1012700094DF811101C026C08CE4F0DE8AE075DFC6
:10128000812FECDE8CE4EADE8BE06FDF81E0E6DECE
:1012900078DF8823B9F081DF8823A1F08BE6DEDEDA
:1012A00084E063DF80EADADE82E0D8DE84E2D6DE44
:1012B000F0DE8883EEDE8983ECDE8A839AB581E0F6
:1012C000911101C080E0DF91CF911F910895CF92DD
:1012D000DF92EF92FF920F931F93CF93DF936B01F7
:1012E0007C01EA01890159DF882361F18CE4B6DED3
:1012F0008AE03BDF83E4B2DE02301105C0F08BE60A
:10130000ADDEC701B60119DF80EAA8DE802F81506B
:10131000A5DE84E2A3DE0C0F1D1F02C0BADE899396
:10132000C017D10759F08AB58111F8CF07C08CE0FA
:1013300095DEC701B60101DFACDE88839AB581E096
:10134000911101C080E0DF91CF911F910F91FF902B
:10135000EF90DF90CF9008950F931F93CF93DF937B
:1013600000D000D0CDB7DEB7182F022F49835A83A3
:101370006B837C8312DF882399F08CE46FDE8AE034
:10138000F4DE812F6BDE8CE469DE49815A816B814A
:101390007C81CB01BA01D1DE802F60DE81E001C00B
:1013A00080E00F900F900F900F90DF91CF911F91E1
:1013B0000F9108952F923F924F925F926F927F927A
:1013C0008F929F92AF92BF92CF92DF92EF92FF9255
:1013D0000F931F93CF93DF93782E662E842E922E39
:1013E00017012801E60120FF11C0D7DE811102C0DC
:1013F00080E042C08CE432DE8AE0B7DE862D2EDE4D
:101400008CE42CDE8BE0B1DE81E028DEA114B10497
:1014100019F491FC1FC02FC0C0DE882349F38CE46F
:101420001DDE8AE0A2DE872D19DE8BE617DEC20103
:10143000B10183DE80EA12DE8A2D81500FDE84E660
:101440000DDEAC0EBD1E02C0899108DECA15DB059B
:10145000D9F7DFCFA2DE882309F4CACF8CE4FEDD02
:101460008AE083DE882DFADD8CE4F8DDC201B1016B
:1014700064DE80E0F3DD81E0DF91CF911F910F9179
:10148000FF90EF90DF90CF90BF90AF909F908F90A4
:101490007F906F905F904F903F902F9008951F9393
:1014A000CF93DF9300D000D0CDB7DEB7182F49839C
:1014B0005A836B837C8371DE49815A816B817C8185
:1014C000882309F467C08CE4103429F4C7DD8AE06E
:1014D0004CDE80E440C049835A836B837C831033A5
:1014E00009F040C0BBDD8AE040DE86E3B7DD8CE476
:1014F000B5DD8BE03ADE81E0B1DD4FDE882309F413
:1015000049C08CE4ABDD8AE030DE83E3A7DD8BE607
:10151000A5DD49815A816B817C81CB01BA010DDE49
:1015200080EA9CDD80917901815098DD84E696DD2A
:1015300010E003C080E092DD1F5F212F30E080913A
:10154000790190917A0128173907A0F38CE486DDA0
:101550008AE00BDE80E382DD8CE480DD8BE005DE5B
:1015600081E00FC07BDD8AE000DE812F77DD8CE437
:1015700075DD49815A816B817C81CB01BA01DDDD4A
:1015800080E06CDD0F900F900F900F90DF91CF9166
:101590001F91F7CD80E00F900F900F900F90DF918B
:1015A000CF911F910895282F207330E0220F331F11
:1015B00020693F6F8F70822B51CD1F93CF93DF93A4
:1015C0001F92CDB7DEB7182F88E6998347DD812FAC
:1015D00045DD89E643DD9981892F0F90DF91CF9119
:1015E0001F913CCD80E83ADD54DD9AB5992321F076
:1015F00081FFF8CF81E0089580E008958091770120
:10160000282F207330E0220F331F20618F70822B30
:1016100025DD3FDD9AB5992321F087FDEFCF81E0ED
:10162000089580E00895BF92CF92DF92EF92FF92EB
:101630000F931F93CF93DF93CDB7DEB728970FB6E5
:10164000F894DEBF0FBECDBF41DD82EC07DD82E046
:1016500005DD80EE03DD7E0189E0E80EF11C8E01E0
:101660000F5F1F4F58E0D52EB02EC12EE9EAF1E0F2
:10167000AB2DBC2D8D2D01900D928A95E1F7F701D0
:1016800082917F01EBDCE016F10681F728960FB618
:10169000F894DEBF0FBECDBFDF91CF911F910F91A8
:1016A000FF90EF90DF90CF90BF909CCF9BDF80ECBE
:1016B000D5DC80E0D3DC80E8D1DCEBDC8111F7CF36
:1016C000B7CCEF92FF920F931F93CF93DF937C01E0
:1016D000EB018A0193DF8823C1F08091780163DFF9
:1016E00080E0BCDCC70169DF0C0F1D1F04C084E271
:1016F000B5DCCFDC8993C017D10719F08AB5811109
:10170000F6CF9AB581E0911101C080E0DF91CF91D1
:101710001F910F91FF90EF900895EF92FF920F931A
:101720001F93CF93DF937C018B01EA0167DF811167
:1017300002C080E023C0C0FF06C0F801EC0FFD1F0F
:101740008FEF80832196809178012DDF8DE186DCFB
:10175000C70133DF10C052DF882359F384E67EDCF3
:10176000F80180817BDC84E679DCF80181810E5F01
:101770001F4F74DC2297209771F781E0DF91CF91A2
:101780001F910F91FF90EF9008951F93CF93DF93D8
:10179000182FEB0133DF882381F08091780103DF7C
:1017A000812F5CDCCE01816008DF80E657DC80E0C1
:1017B00055DCDF91CF911F9121CF80E0DF91CF9158
:1017C0001F910895BF92CF92DF92EF92FF920F93F5
:1017D0001F93CF93DF937C018B01EA0173D2B82E64
:1017E000811133C0209731F028813981021B130BFE
:1017F000E20EF31EC12CD12C23C08091E80085FDA0
:1018000015C08091E8008E778093E800FBD4209784
:1018100049F0888199818C0D9D1D9983888325E0ED
:10182000B22E13C04FD2882359F00EC0F701819118
:101830007F018093F10001501109FFEFCF1ADF0AF9
:1018400001151105D1F601C0B82E8B2DDF91CF9176
:101850001F910F91FF90EF90DF90CF90BF90089570
:10186000BF92CF92DF92EF92FF920F931F93CF938D
:10187000DF937C018B01EA0125D2B82E811133C0A0
:10188000209731F028813981021B130BE20EF31EE1
:10189000C12CD12C23C08091E80085FD15C080911A
:1018A000E8008B778093E800ADD4209749F08881D9
:1018B00099818C0D9D1D9983888345E0B42E13C0BA
:1018C00001D2882359F00EC08091F100F701819375
:1018D0007F0101501109FFEFCF1ADF0A0115110531
:1018E000D1F601C0B82E8B2DDF91CF911F910F91B2
:1018F000FF90EF90DF90CF90BF900895BF92CF926E
:10190000DF92EF92FF920F931F93CF93DF936C01BF
:101910008B017A01D7D1B82E81113AC0E801219705
:10192000CC0DDD1DE114F10439F0F7012081318186
:10193000021B130BC21BD30BC12CD12C24C08091D2
:10194000E80085FD17C08091E8008B778093E80060
:1019500059D4E114F10451F0F701808191818C0D8B
:101960009D1D9183808355E0B52E12C0ABD1882395
:1019700051F00DC08091F100888321970150110929
:10198000FFEFCF1ADF0A01151105C9F601C0B82E05
:101990008B2DDF91CF911F910F91FF90EF90DF90F2
:1019A000CF90BF9008952091E8023091E902261768
:1019B000370748F06115710539F42091E8002E775A
:1019C0002093E80001C0B901FC0120E02BC08EB3D8
:1019D0008823D9F18530D9F18091E80083FD33C0A7
:1019E0008091E80082FD29C08091E80080FF1AC044
:1019F0008091F2009091F30006C021912093F100B4
:101A00006150710901966115710519F080319105D8
:101A1000A0F321E0409709F020E08091E8008E7764
:101A20008093E8006115710591F62111D0CF05C0B2
:101A30008EB3882351F0853051F08091E80082FF09
:101A4000F7CF80E0089581E0089582E0089583E073
:101A500008952091E8023091E9022617370748F0EF
:101A60006115710539F42091E8002E772093E80084
:101A700001C0B901FC0120E02EC08EB3882309F417
:101A80003DC0853009F43CC08091E80083FD34C03E
:101A90008091E80082FD2AC08091E80080FF1BC091
:101AA0008091F2009091F30007C024912093F100FF
:101AB00031966150710901966115710519F08031F7
:101AC000910598F321E0409709F020E08091E8002B
:101AD0008E778093E8006115710579F62111CDCFDD
:101AE00005C08EB3882351F0853051F08091E80015
:101AF00082FFF7CF80E0089581E0089582E00895A5
:101B000083E00895EF92FF920F931F93CF93DF939B
:101B1000EB012091E8023091E9022617370740F0E7
:101B2000209739F42091E8002E772093E80001C037
:101B3000E9019C0180E038C09EB3992309F446C0B6
:101B4000953009F445C09091E80093FD3DC0909117
:101B5000E80092FD33C09091E80090FF25C000910D
:101B6000F2001091F3007901E01AF10A07C0CA01EE
:101B7000F4D48093F10021970F5F1F4FA701400F0E
:101B8000511F742F652F209719F00031110578F33C
:101B900081E00031110509F080E09091E8009E7726
:101BA0009093E800272F362F209731F68111C4CF6C
:101BB00005C08EB3882351F0853051F08091E80044
:101BC00082FFF7CF80E005C081E003C082E001C062
:101BD00083E0DF91CF911F910F91FF90EF900895D7
:101BE0008F708093E900EBEEF0E08081816080836C
:101BF000EDEEF0E010826093EC0040838091EE0007
:101C0000881F8827881F08950F931F93CF93DF9312
:101C1000062FEC0110E02FC09881911103C01F5FC7
:101C2000259629C02C81E981FA817B81892F8F70CB
:101C3000873010F080E022C0223010F056E001C062
:101C400052E028E030E040E003C04F5F220F331F36
:101C50002E173F07D0F34295407F452B692F661F13
:101C60006627661F90E4799F90011124622BB8DFEC
:101C70008111D5CFDFCF1013CFCF81E0DF91CF918E
:101C80001F910F9108958091E20287FD05C0809118
:101C9000E80080FF0DC010C08091E80082FD04C004
:101CA0008EB38111F9CF08958091E8008B7707C03A
:101CB0008EB38111ECCF08958091E8008E778093E8
:101CC000E80008958091E4009091E50045E62091B8
:101CD000EC0020FD1EC022C02EB3222391F025303F
:101CE00091F02091EB0025FD10C02091E40030918F
:101CF000E5002817390759F34150C90141F784E03D
:101D0000089582E0089583E0089581E0089580E0D9
:101D100008952091E80020FFDFCFF9CF2091E8005F
:101D200022FFDACFF4CF0F931F93CF93DF9349D0E5
:101D300050D0C8EDD0E088818F7788838881806813
:101D4000888388818F7D8883E7EDF0E080818068DB
:101D5000808319BC1EBA1092E00200EE10E0F80178
:101D600080818B7F808388818160888342E160E00D
:101D700080E036DFE1EEF0E080818E7F8083E2EE6E
:101D8000F0E0808181608083808188608083F801B9
:101D900080818E7F8083888180618883DF91CF916D
:101DA0001F910F910895E8EDF0E080818F7E808390
:101DB000E7EDF0E080818160808381E08093E10243
:101DC000B2CFE8EDF0E080818C7F80831092E2005A
:101DD00008951092DA001092E10008951F920F9278
:101DE0000FB60F9211240BB60F922F933F934F9380
:101DF0005F936F937F938F939F93AF93BF93EF9373
:101E0000FF938091DA0080FF1DC08091D80080FF91
:101E100019C08091DA008E7F8093DA008091D9001A
:101E200080FF0CC08CE089BD8EE089BD09B400FE46
:101E3000FDCF81E08EBB0E94FF0104C019BC1EBA19
:101E40000E9401028091E10080FF17C08091E200B2
:101E500080FF13C08091E2008E7F8093E20080912A
:101E6000E20080618093E2008091D80080628093DC
:101E7000D80019BC85E08EBBC4D18091E10084FFFD
:101E80002EC08091E20084FF2AC08CE089BD8EE0E4
:101E900089BD09B400FEFDCF8091D8008F7D80936D
:101EA000D8008091E1008F7E8093E1008091E20074
:101EB0008F7E8093E2008091E20081608093E20057
:101EC0008091E002882311F084E007C08091E30054
:101ED00087FF02C083E001C081E08EBB92D1809178
:101EE000E10083FF21C08091E20083FF1DC080914B
:101EF000E100877F8093E10082E08EBB1092E002D8
:101F00008091E1008E7F8093E1008091E2008E7FDE
:101F10008093E2008091E20080618093E20042E1E0
:101F200060E080E05DDE6DD1FF91EF91BF91AF91F8
:101F30009F918F917F916F915F914F913F912F91E1
:101F40000F900BBE0F900FBE0F901F9018951F9310
:101F5000CF93DF93CDB7DEB7AD970FB6F894DEBF62
:101F60000FBECDBFE2EEF2E08091F100819322E05E
:101F7000EA3EF207C9F70E94F6018091E80083FF6C
:101F800028C18091E2029091E302953009F470C07B
:101F900038F4913079F170F0933009F01AC12AC009
:101FA000983009F4E8C0993009F4F7C0963009F088
:101FB00010C183C0803899F0823809F00AC180913D
:101FC000E6029091E7028F7099278093E900909143
:101FD000EB0095FB992790F91092E90001C090E081
:101FE0008091E800877F8093E8009093F100109241
:101FF000F100CCC0882319F0823009F0EAC08F715B
:10200000823009F0E6C08091E40281112BC08091FA
:10201000E6029091E7028F709927009709F4D9C0E2
:102020008093E9002091EB0020FF1CC02091E30287
:10203000233021F48091EB00806212C09091EB007C
:1020400090619093EB0021E030E001C0220F8A956F
:10205000EAF72093EA001092EA008091EB00886092
:102060008093EB001092E9008091E800877F91C097
:102070008111AFC08091E4029091E5028F7799279A
:10208000182F9091E3009078982B9093E300809123
:10209000E800877F8093E800F6DD8091E80080FF0C
:1020A000FCCF8091E30080688093E300112311F05E
:1020B00083E001C082E08EBB8CC08058823008F083
:1020C00088C08091E4029091E5028C3D23E0920764
:1020D00069F583E08A838AE289834FB7F894DE0149
:1020E000139620E03EE051E2E32FF0E050935700DA
:1020F000E49120FF03C0E295EF703F5FEF708E2FF9
:1021000090E0EA3010F0C79601C0C0968D939D9381
:102110002F5F243149F74FBF8091E800877F80937C
:10212000E8006AE270E0CE0101961EC09E01235DC8
:102130003F4FAE01455D5F4F6091E6020E9419027C
:10214000BC01009709F445C08091E800877F809327
:10215000E8002DA58BA59CA5211102C07ADC05C045
:10216000213011F4CFDC01C01EDC8091E8008B77B8
:102170008093E8002EC0803861F58091E800877F69
:102180008093E8008091E0028093F1008091E80064
:102190008E778093E80077DD1CC081111AC0909182
:1021A000E4029230B0F48091E800877F8093E800E9
:1021B0009093E00268DD8091E002811104C080917B
:1021C000E30087FF02C084E001C081E08EBB0E9473
:1021D000A7018091E80083FF0AC08091E800877F13
:1021E0008093E8008091EB0080628093EB00AD96D5
:1021F0000FB6F894DEBF0FBECDBFDF91CF911F9118
:1022000008950895CF938EB38823A9F08091E900B3
:102210008F709091EC0090FF02C090E801C090E0B8
:10222000C92FC82B1092E9008091E80083FD8FDE52
:10223000CF70C093E900CF910895CF93DF93EC0165
:102240004096FC018BE0DF011D928A95E9F782E060
:102250008C83898783E08E8761E0CE010196D4DC90
:10226000882361F061E0CE010696CEDC882331F050
:1022700061E0CE010B96DF91CF91C6CC80E0DF917B
:10228000CF910895CF93C62F2EB32430F1F4FC01E3
:102290004489558966897789452B462B472BA9F0B8
:1022A00081818F708093E9008091E80085FF04C0F0
:1022B000C093F10080E00AC08091E8008E7780939F
:1022C000E80000DD8823A1F301C082E0CF910895EA
:1022D0002EB3243039F5FC01448955896689778904
:1022E000452B462B472BF1F081818F708093E900BD
:1022F0008091F2009091F300892B11F480E0089511
:102300009091E8008091E8008E778093E80095FD39
:10231000F5CFD8DC811107C09091E8009E779093AB
:10232000E800089582E008952EB3243089F4FC017A
:102330004489558966897789452B462B472B41F07F
:1023400021812F702093E9002091E80020FDC0CF6B
:1023500008952EB3243019F02FEF3FEF28C0FC0171
:102360004489558966897789452B462B472BA1F3EC
:1023700086818F708093E9008091E80082FFECCF26
:102380008091F2009091F300892B21F02091F100CF
:1023900030E002C02FEF3FEF8091F2009091F30008
:1023A000892B29F48091E8008B778093E800C9019C
:1023B00008950895CF93DF93EC018091E80083FFA7
:1023C000A7C0888190E02091E6023091E7022817AB
:1023D000390709F09DC08091E302813261F020F459
:1023E000803209F095C03DC0823209F46DC083325D
:1023F00009F08EC07DC08091E202813A09F088C068
:102400008091E800877F8093E8008091E80080FF5A
:10241000FCCF4C895D896E897F894093F100BB2791
:10242000A72F962F852F8093F100CB01AA27BB27DA
:102430008093F100472F5527662777274093F100B7
:10244000888D8093F100898D8093F1008A8D80932F
:10245000F1008091E8008E778093E800DF91CF91C2
:1024600012CC8091E202813209F052C08091E800E2
:10247000877F8093E80004C08EB3882309F448C0A6
:102480008091E80082FFF8CF3091F1002091F100B7
:102490009091F1008091F1003C8B2D8B9E8B8F8B66
:1024A0008091F100888F8091F100898F8091F100F7
:1024B0008A8F8091E8008B778093E800E4DBCE017F
:1024C000DF91CF910C9403028091E202813201F5F9
:1024D0008091E800877F8093E800D5DB8091E4025B
:1024E0009091E502998B888BCE01DF91CF9161CFDE
:1024F0008091E202813261F48091E800877F8093CD
:10250000E800C1DB6091E402CE01DF91CF9151CFB1
:10251000DF91CF910895A1E21A2EAA1BBB1BFD01EA
:102520000DC0AA1FBB1FEE1FFF1FA217B307E407B2
:10253000F50720F0A21BB30BE40BF50B661F771F0A
:10254000881F991F1A9469F76095709580959095EA
:102550009B01AC01BD01CF010895F999FECF92BD59
:1025600081BDF89A992780B50895262FF999FECF55
:1025700092BD81BDF89A019700B4021639F01FBAD6
:1025800020BD0FB6F894FA9AF99A0FBE0895F89400
:02259000FFCF7B
:102592000083100000010410000001820800000105
:1025A20000000000000000000000001C03300030AA
:1025B2000030003200300030003000310032003391
:1025C2000034003500000000000902200001010073
:1025D200C0320904000002FF000000070582024029
:1025E200000A0705020240000A80010081010090F2
:1025F20001009101019201179401219803069E03A3
:1026020001A10110A4030032332000C001000140E7
:10261200206830222A3218242C354C081A232333FE
:10262200232323262636262626010101000001380F
:10263200391289AB45CDD888FF1289AB45CDD888F0
:0C264200FF4156524953505F4D4B32008F
:00000001FF
